:100000000C94E4010C941C020C941C020C941C0231
:100010000C941C020C941C020C941C020C941C02E8
:100020000C941C020C941C020C940E200C94E020E6
:100030000C94ED1A0C941C020C941C020C941C02DF
:100040000C941C020C941C020C941C020C941C02B8
:100050000C941C020C94751B0C941C020C941C0236
:100060000C941C020C941C020C941C020C941C0298
:100070000C941C020C941C020C941C020C941C0288
:100080000C941C020C941C020C941C020C941C0278
:100090000C941C020C941C020C941C020C941C0268
:1000A0000C941C020C941C020C941C02F404F40426
:1000B000200520058805A605BE06BE06B1054A0630
:1000C0005B065B064D2174216C2274216C22C021D9
:1000D000E3216C223A22492229003A003B003C00ED
:1000E0003D0000003E003F00400041004200430050
:1000F0004400450000004C0035001E001F00200099
:1001000021002200230024002500260027002D00C6
:100110002E004C002A004A002B00000014001A0098
:100120000800150017001C0018000C001200130036
:100130002F00300031004B00390000000400160091
:10014000070009000A000B000D000E000F0033002D
:100150003400280000004E00E10064001D001B0078
:1001600006001900050011001000360037003800A5
:100170000000E50052004D00E000E3000000E20056
:10018000000000002C00000000000000E60001510B
:10019000E400500051004F00010001000100010087
:1001A0000100000001000100010001000100010048
:1001B0000100010000000100010001000100010038
:1001C0000100010001000100010001000100010027
:1001D00001000100005C01000100000001000100BD
:1001E0000100010001000100010001000100010007
:1001F00001000100010001000100000001000100F8
:1002000001000100010001000100010001000100E6
:1002100001000100000001000100010001000100D7
:10022000BE5CC05CBF5CC15C01000100010001005C
:1002300000000100010001000100010000000100B8
:1002400000000000010000000000000001000100AB
:10025000010001000100010012035000720069005A
:100260006D007500730037003500000012036D004B
:100270006F0079006900340036003800310000005A
:100280000403090409023B00020100A0FA0904006A
:1002900000010301010009211101000122400007B2
:1002A00005810308000109040100010300000009A1
:1002B000211101000122B60007058203200001126E
:1002C000010002000000085A44141001000102005D
:1002D0000105010902A10185020901A10005091911
:1002E00001290815002501950875018102050109FC
:1002F0003009311581257F95027508810609381569
:1003000081257F950175088106050C0A3802158143
:10031000257F950175088106C0C005010980A101EE
:10032000850319012AB700150126B700950175103C
:100330008100C0050C0901A101850419012AA00250
:10034000150126A002950175108100C0050109065E
:10035000A1018506050719E029E715002501950883
:10036000750181020507190029EF1500250195F097
:10037000750181020508190129059505750191028C
:10038000950175039101C005010906A10105071931
:10039000E029E71500250195087501810295017591
:1003A0000881010507190029FF150026FF009506A1
:1003B0007508810005081901290595057501910247
:1003C000950175039101C00011241FBECFEFDAE043
:1003D000DEBFCDBF04B603FE18C08091D802909155
:1003E000D902A091DA02B091DB028730904BA7408E
:1003F000B04B59F41092D8021092D9021092DA023E
:100400001092DB02E0E0F8E3099511E0A0E0B1E032
:10041000E6EDF6E402C005900D92A239B107D9F7D6
:1004200022E0A2E9B1E001C01D92A83DB207E1F7C8
:100430000E94CE120C9469230C94000081E0089570
:1004400081E008950C94200208950C9424021F93D7
:10045000CF93DF9300D000D01F92CDB7DEB7498392
:100460005A836B833091950189819A81311114C02F
:10047000662359F0222349F00E94FB08182F682FA9
:1004800089819A810E94A40803C00E94CF08182F76
:1004900069817A81812F04C00E94FB0869817A8179
:1004A0000F900F900F900F900F90DF91CF911F91B1
:1004B0000C943710FC01262F408151816281738199
:1004C00084810C94270281E00895CF93DF93EC019F
:1004D00060E00E945A02BE01DF91CF910C94250288
:1004E0000C947F110C947B1108950E944E070E947A
:1004F00074022FEF84E39CE0215080409040E1F7AC
:1005000000C000000C949B1B0F931F93CF93DF93AD
:100510008C0161E00E945A02EC01B8010E942202A3
:10052000882309F444C0B801CE010E9451168823E3
:10053000F1F1B801CE010E9438198823C1F1B80148
:10054000CE010E944C17882391F1B801CE010E9480
:100550009418882361F1F8018281882309F1CB3551
:100560008DE5D807C1F050F4C115FCE5DF0781F037
:10057000CF3DDC45A9F40E94320E19C0CC35EDE523
:10058000DE0761F0CD35DD4559F40E94750D08C0D8
:100590000E9475020CC00E947E0D02C00E94810D57
:1005A000C801DF91CF911F910F910C941E0280E042
:1005B000DF91CF911F910F9108950E94CF1A80E093
:1005C0000E9486160C9417030E9475150E941A0348
:1005D0000C94D51A08950C94EA0281E00895CF9303
:1005E000C82F0E94ED02882381F0C095C0FF02C091
:1005F000729A01C07298C1FF02C02A9A01C02A985B
:10060000C2FF02C08F9A01C08F98CF9108956A9A55
:10061000729A229A2A9A879A8F9A0895CF93C82F0E
:100620000E94EB028C2F0E94EF02CF91089580E090
:100630000C940E030E9494190C940E030E949419BA
:1006400090919401891721F0809394010C940E03EA
:100650000895CF93DF93CDB7DEB72B970FB6F894FD
:10066000DEBF0FBECDBF4F83588769877A878B87E0
:1006700061110E94C10C9E012F5F3F4F86E0F9017E
:1006800011928A95E9F785E0FE013796D90101902C
:100690000D928A95E1F789819A814C815D81452B84
:1006A00031F09F3F31F491E08F3F19F403C091E0A6
:1006B00001C090E090FF09C049815A816B817C8123
:1006C0008D819E810E94E20B05C0C9010E946302D8
:1006D0008111F2CF2B960FB6F894DEBF0FBECDBFBF
:1006E000DF91CF910895FC01808191810E943D09A5
:1006F0000895CF93882309F4A4C0C82F8238C1F489
:100700000E94941981FD9DC069E38091020190913E
:1007100003010E948A1A0E94E30C2FEF81EE94E0FD
:10072000215080409040E1F700C0000069E319C00B
:10073000833801F50E94941980FD83C063E58091A0
:100740000201909103010E948A1A0E94E30C2FEF8C
:1007500081EE94E0215080409040E1F700C000001D
:1007600063E580910201909103010E94951ACF9157
:100770000C94E30C8438C1F40E94941982FD61C08A
:1007800067E480910201909103010E948A1A0E94FD
:10079000E30C2FEF81EE94E0215080409040E1F790
:1007A00000C0000067E4DDCF8CEF8C0F813AD0F4FD
:1007B0006C2F80910201909103010E940A1A8823F4
:1007C00049F06C2F80910201909103010E94951ACB
:1007D0000E94E30C6C2F80910201909103010E9412
:1007E0008A1AC5CF80E28C0F883048F4C77081E048
:1007F00001C0880FCA95EAF70E94A40CB8CFEBE5B8
:10080000EC0FE33040F4F0E0E95BFE4F808190E0D4
:10081000CF910C94C819E8E5EC0FE73150F4F0E003
:10082000EE0FFF1FE75EFE4F80819181CF910C9408
:10083000DE19CD3E30F08C2F0E945313CF910C94D3
:100840002514CF910895882309F464C0823879F47F
:100850000E94941981FF5EC069E38091020190912A
:1008600003010E948A1A0E94E30C69E310C08338D6
:10087000B1F40E94941980FF4DC063E5809102019C
:10088000909103010E948A1A0E94E30C63E5809113
:100890000201909103010E94951A0C94E30C843894
:1008A00079F40E94941982FF35C067E480910201B7
:1008B000909103010E948A1A0E94E30C67E4E7CF3B
:1008C0009CEF980F913A10F4682FE1CF90E2980FC7
:1008D000983050F4877091E001C0990F8A95EAF73B
:1008E000892F0E94AA0CD9CF9BE5980F933020F452
:1008F00080E090E00C94C81998E5980F973120F4A7
:1009000080E090E00C94DE198D3E20F00E94AE1342
:100910000C94251408951F93CF93DF93182FEB01A8
:100920000E947903209741F08FE99FE00197F1F74A
:1009300000C000002197F6CF812FDF91CF911F914A
:100940000C942304893319F060E070E002C060E584
:1009500070E00C948B04882321F00E94A40C0C946A
:10096000E30C0895882321F00E94AA0C0C94E30C58
:100970000895CF92DF92EF92FF920F931F93CF9340
:10098000DF937C01D62FC72FFC01128105810295D0
:100990000F700E949A0C8823B9F01123A9F08C2FB4
:1009A000807F803421F080E28D0F883068F0809164
:1009B000AD0282FD09C082E00E94430D0E949A0CA4
:1009C00091E0D82ED92601C0D12CCC2EC2948FE034
:1009D000C8228C2D90E08C30910508F0CFC1FC012D
:1009E000EA5AFF4F0C94FA228C2F807FCF70882315
:1009F00011F0C295C07F112399F0CC2309F4AAC14C
:100A000080E28D0F883010F0D11104C08C2F0E942D
:100A1000A40C03C08C2F0E94B40C0E94E30C9AC15A
:100A20008D2F0E942304CC2309F4A8C180E28D0FEE
:100A3000883038F1DD2329F18C2F0E94BA0C24C0B4
:100A40008C2F807FCF70803211F0C295C07FDD2364
:100A500019F0D130A1F13DC08091AD0282FF17C0E5
:100A6000112349F0CC2329F08C2F0E94A40C0E9462
:100A7000E30C80E070C180E00E942304CC2309F4E1
:100A80007DC18C2F0E94AA0C0E94E30C77C1112318
:100A900071F0002341F0013031F40E94C40C8C2B22
:100AA0000E94CC0C6BC10E94C40C8C2B1DC0002377
:100AB00019F0013009F462C10E94D90C25C011233C
:100AC00021F0063008F05AC10EC0053008F056C1BA
:100AD0001BC0112361F0002331F0F701858180FFF5
:100AE00039C18F7085838C2F0E94AB0447C10023CE
:100AF00059F0D93309F03FC1FFEF07EE13E0F15091
:100B000000401040E1F735C18C2F0E94B20436C17D
:100B10008C2F86958695837019F0813061F02EC1F7
:100B2000112321F08D2F9C2F937002C080E090E064
:100B30000E94C8192BC1112321F08D2F9C2F937077
:100B400002C080E090E00E94DE1920C18D2F1123A9
:100B500019F00E94531302C00E94AE130E94251484
:100B600015C18C2F837009F047C011110BC12D2FB7
:100B7000229526952770220F220F6D2F6F70862FDA
:100B800090E0A0E0B0E0022E04C0880F991FAA1FD9
:100B9000BB1F0A94D2F7D4FF10C04FE050E060E0D2
:100BA00070E004C0440F551F661F771F2A95D2F7C7
:100BB000409550956095709503C040E050E0BA01B3
:100BC000C695C695C3708A019B01082B192B2A2B49
:100BD0003B2BC901B801C23049F058F4C13019F0BB
:100BE0000E94BA07CFC00E94A807CCC00E94CC07C1
:100BF000C9C00E94A607C6C0112319F08C2F8170AE
:100C000001C08695882309F4BDC02D2F2295269515
:100C10002770220F220F6D2F6F70862F90E0A0E0BB
:100C2000B0E0022E04C0880F991FAA1FBB1F0A94B0
:100C3000D2F7D4FF10C04FE050E060E070E004C095
:100C4000440F551F661F771F2A95D2F74095509580
:100C50006095709503C040E050E0BA01C695C69516
:100C6000C3708A019B01082B192B2A2B3B2BC9012E
:100C7000B801C23049F058F4C13019F00E947F0821
:100C800081C00E946D087EC00E9491087BC00E94B6
:100C9000E00778C0CF70112339F08C2F0E9406082E
:100CA0008D2F0E94AB046EC08D2F0E94B2048C2F3A
:100CB0000E94270867C0D23F21F128F4D03F41F0BD
:100CC000D13FC1F043C0D33F19F1D43F79F03EC0CA
:100CD000112341F0053008F051C08C2F8F710E9414
:100CE0004C084CC0063008F049C0F7CF8091AD02E7
:100CF00082FF18C0112339F08C2F8F710E940608D3
:100D00003DC01123C9F38C2F8F710E94270836C074
:100D1000112329F08C2F8F710E94F1072FC00E94A0
:100D2000EC072CC0112349F0CF718C2F0E940608CC
:100D300063E08C2F0E94280D21C081E00E94430DAA
:100D40000230E0F082E00E94430D18C0112331F020
:100D5000002391F28D2F0E94790310C0002399F295
:100D6000D93349F41FEF27EE33E0115020403040D3
:100D7000E1F700C000008D2F0E94230488EF8C0D46
:100D8000843020F40E9494190E940E03DD20C9F0E3
:100D90000E94960C80FD15C0F70112820E94900CF3
:100DA0000E940608C7010E9402070E94900CDF9172
:100DB000CF911F910F91FF90EF90DF90CF900C9407
:100DC0002708DF91CF911F910F91FF90EF90DF9057
:100DD000CF9008950F931F93CF93DF93EC01688119
:100DE00079818A810E9448098C010E94A3080E948F
:100DF0009407B801CE010E94B904DF91CF911F91F1
:100E00000F910895CF93DF93EC01988189812B8115
:100E10003C81232B31F08F3F31F481E09F3F19F467
:100E200003C081E001C080E080FD1DC0CE010E94B2
:100E30008402811110C00E949A0C8823A1F08A813B
:100E4000882389F08091AD0282FD0DC082E0DF91A0
:100E5000CF910C94430DCE010E94EA06CE01DF91A2
:100E6000CF910C946502DF91CF91089580E090E0DE
:100E70000E94C81980E090E00E94DE190E94C10C17
:100E80000E94E30C0E9456150C94251480910201D7
:100E9000909103010E94A01A0C9436070E94B10C95
:100EA0000C94460792959F70963079F010F492500A
:100EB00001C09A50923068F4803F69F018F4883E7F
:100EC00040F409C0843F29F406C0883E20F0813FE9
:100ED00011F080E0089581E00895FC018081918106
:100EE0000E943D090E9452070895CF93DF9300D0DE
:100EF00000D01F92CDB7DEB70F900F900F900F90DC
:100F00000F90DF91CF910895CF93DF9300D000D061
:100F100000D0CDB7DEB726960FB6F894DEBF0FBE71
:100F2000CDBFDF91CF910895089508950C94950752
:100F30000C9496070E9498076093D6017093D7018E
:100F40008093D8019093D9010C9436070C949A079A
:100F50000F931F930091D6011091D7012091D801D2
:100F60003091D901602B712B822B932B1F910F9104
:100F70000C949A070F931F930091D6011091D701FB
:100F80002091D8013091D9016023712382239323CA
:100F90001F910F910C949A070F931F930091D60104
:100FA0001091D7012091D8013091D9016027712784
:100FB000822793271F910F910C949A070C94950701
:100FC0000E94DE076093D2017093D3018093D40115
:100FD0009093D5010C94360760E070E0CB010C943F
:100FE000E0070F931F9341E050E060E070E08A015A
:100FF0009B0104C0000F111F221F331F8A95D2F7D7
:10100000C901B8011F910F910C94E0070F931F9332
:1010100041E050E060E070E004C0440F551F661FDF
:10102000771F8A95D2F78091D2019091D301A09138
:10103000D401B091D5018A019B01082B192B2A2BD1
:101040003B2BC901B8011F910F910C94E0070F933E
:101050001F9341E050E060E070E004C0440F551F72
:10106000661F771F8A95D2F74095509560957095C9
:101070008091D2019091D301A091D401B091D5017A
:101080008A019B01082319232A233B23C901B801A4
:101090001F910F910C94E0070F931F9341E050E0D4
:1010A00060E070E004C0440F551F661F771F8A95EB
:1010B000D2F78091D2019091D301A091D401B09147
:1010C000D5018A019B01082719272A273B27C90137
:1010D000B8011F910F910C94E0070F931F9300919B
:1010E000D2011091D3012091D4013091D501602B10
:1010F000712B822B932B1F910F910C94E0070F9370
:101100001F930091D2011091D3012091D40130910D
:10111000D50160237123822393231F910F910C9497
:10112000E0070F931F930091D2011091D3012091FA
:10113000D4013091D50160277127822793271F9111
:101140000F910C94E007089520E1929F800D1124E7
:10115000E82FE695E695E695877051E001C0550FBA
:101160008A95EAF785E0E89FF0011124EA56FE4FE0
:1011700020E030E070E04081CB01022E02C0969565
:1011800087950A94E2F781708195842785238427C7
:1011900081932F5F3F4F2530310569F7089520E196
:1011A000929F800D1124682F669566956695982FFD
:1011B000977085E0689FB001112440E050E080E026
:1011C000FB01E40FF51FEA56FE4F208130E0092EA7
:1011D00002C0369527950A94E2F721703327042E32
:1011E00001C0220F0A94EAF7822B4F5F5F4F453010
:1011F000510531F70895BF92CF92DF92EF92FF929F
:101200000F931F93CF93DF938C01C090D201D090A6
:10121000D301E090D401F090D5018091D601909156
:10122000D701A091D801B091D901C82AD92AEA2AB8
:10123000FB2ACFE1D0E0D701C6010C2E04C0B69541
:10124000A795979587950A94D2F780FD04C02197BA
:1012500090F7B12C07C0BC2EB8018C2F0E944C1007
:101260000197A9F38B2DDF91CF911F910F91FF90E3
:10127000EF90DF90CF90BF900895CF93DF93EC0174
:101280000E94FB08BE010E944C10DF91CF9108958F
:101290001F93CF93DF93EB0190919501992321F058
:1012A000CB010E943D0913C0882349F0CB010E9465
:1012B000FB08182F682FCE010E94A40804C0CB01A0
:1012C0000E94CF08182FBE01812F0E944C10DF9181
:1012D000CF911F9108951F93CF93DF93C091DA01AF
:1012E00016E08091DB01C81799F0D0E01C9FF00157
:1012F0001D9FF00D1124E452FE4F40815181628107
:101300007381848195810E9484072196C770E9CFFB
:10131000DF91CF911F91089540910C0250910D02E1
:1013200060910E0270910F02809110029091110253
:101330000C948407EF92FF920F931F93CF93DF9348
:101340008091110282958F7009F065C080910E0224
:10135000882309F460C08091DA01F090DB011091DC
:101360000C0200910D0260910F027091100291E049
:101370001F3F09F090E0C0910001D0910101292F99
:1013800096E0E92E8F1509F446C06115710521F02C
:101390000F3F21F030E003C031E001C0322F90E078
:1013A00030FD36C0E89EF001E99EF00D1124DF010A
:1013B000A452BE4F11963C911197301329C03C9115
:1013C000311326C012963C911297311121C0139609
:1013D0004D915C911497461B570B4C175D07C0F459
:1013E000809111028F70806180931102EF51FE4F46
:1013F00080818F70806180838CE092E00E94020780
:10140000DF91CF911F910F91FF90EF900C946B099A
:1014100001968770B7CFDF91CF911F910F91FF9009
:10142000EF9008959F92AF92BF92CF92DF92EF928A
:10143000FF920F931F93CF93DF93CDB7DEB76197E2
:101440000FB6F894DEBF0FBECDBF8C0185E0F8016A
:10145000DE011D9601900D928A95E1F7D801129652
:10146000EC9090910C02E0910D0220910F023091CE
:1014700010022115310531F0EF3F31F481E09F3F3B
:1014800019F403C081E001C080E0B82FB1709B2E39
:1014900080FD47C1D8014C9111965C91119713962C
:1014A000AD90BC9014978CE0C82E82E0D82EF090BE
:1014B0000E02B501621B730B2091000130910101F6
:1014C000FF2009F4D9C0809111026217730708F058
:1014D00095C0282F207F09F052C05E1313C0491316
:1014E00011C0FE2CE1100EC08F708061809311023C
:1014F0000E948C09C6010E94020780911102F80126
:1015000085834DC1AB2831F05F3F31F481E04F3F1F
:1015100019F403C081E001C080E080FD03C081E0D8
:101520008E2502C080E090E0F82FF170FF2E80FF42
:101530001CC08091DA012091DB0136E0821709F4AA
:101540000BC190E0389FF001399FF00D1124E45257
:10155000FE4F6181561306C06081461303C062814D
:10156000E61203C001968770E9CFFE2CEE2009F445
:1015700016C18091110281608093110254C05E13E4
:1015800006C0491304C0E11002C0F80199C0C801A7
:101590000E946D07882361F1EE2051F12091110224
:1015A000822F82958F7090E0029774F080910C02E8
:1015B00090910D0298878F831986BB86AA862C8707
:1015C000CE0107960E94020786E0F801ACE0B2E087
:1015D00001900D928A95E1F70E949A090E948C0968
:1015E0000AC05E1711F1C8010E946D0781112CC05D
:1015F000C8010E940207FF24F394D1C0282F207F46
:1016000081F77A2DB98AA88A6E2D89890E9475077B
:101610008CE092E00E94020786E0D6011D928A9536
:10162000E9F70E948C09F12CBAC04913DCCFE11014
:10163000DACFF8018583C8010E94020786E0D6014F
:101640001D928A95E9F7ABC0EE2091F2209111022C
:10165000822F82958F7090E002970CF4B5CF809125
:101660000C0290910D029A8389831B82BD82AC8209
:101670002E83CE010196A6CF6217730708F044C0EF
:10168000FE2CEE2009F4B4CF5E1330C049132EC0F7
:101690002091110220FD21C0822F82958F70482F4A
:1016A00050E041155105C9F0F80125834F3051052F
:1016B00041F08F5F982F9295907F822F8F70892BAA
:1016C0008583C8010E94020786E0F801ACE0B2E021
:1016D00001900D928A95E1F73CC086E0F801ACE0FC
:1016E000B2E001900D928A95E1F759C0C8010E94BD
:1016F0006D07811169CF8091110281608093110281
:10170000C8010E9402074BC07A2DB98AA88A6E2DA3
:1017100089890E94750786E0D6011D928A95E9F7AE
:1017200018C0EE2009F464CFC8010E946D07F82E9E
:10173000882309F45DCF86E0F801ACE0B2E00190C7
:101740000D928A95E1F78CE092E00E9473030E946B
:101750009A090E948C0923C04D875E878D859E85DE
:101760000E943D09292F22952F70223028F49F7066
:1017700039F0811105C00BC0243028F49F7049F462
:10178000805E883020F0C8010E9402079F2CF92C4F
:1017900006C0D80115969C91907F91F7F8CF8F2DB8
:1017A00061960FB6F894DEBF0FBECDBFDF91CF912B
:1017B0001F910F91FF90EF90DF90CF90BF90AF906F
:1017C0009F9008951F93CF93DF93CDB7DEB72C97EB
:1017D0000FB6F894DEBF0FBECDBF4F835887698721
:1017E0007A878B879C87CE0107960E94120A8823EE
:1017F000D1F09F8188852A853B85232B31F08F3F4F
:1018000031F481E09F3F19F403C081E001C080E022
:1018100080FD47C04F81588569857A858B859C8579
:101820000E9484073EC086E0FE013796DE011196D5
:1018300001900D928A95E1F7FF81E8856A857B85A5
:101840006115710531F0EF3F31F481E0FF3F19F48C
:1018500003C081E001C080E080FD23C02091DB0156
:1018600030E0C9010196877099274091DA0150E074
:1018700084179507F1F1F983EA837D836C8396E001
:10188000929FD001939FB00D1124A452BE4FFE0130
:10189000319601900D929A95E1F78093DB010E94B9
:1018A0006B0916E08091DA019091DB01891771F1E3
:1018B000189FC001112484529E4F0E94120A88234F
:1018C00029F1E091DA011E9FF0011124E452FE4F4C
:1018D0004081518162817381848195810E94840756
:1018E0008091DA0190E00196877099278093DA0160
:1018F000D9CF0E944E071092DB011092DA01ECE082
:10190000F2E086E0DF011D928A95E9F72C960FB68A
:10191000F894DEBF0FBECDBFDF91CF911F91089528
:101920008091320285958595859508958091320242
:101930008770089590913202977081E009F480E0F9
:10194000089580915502089590915502892B8093B6
:1019500055020895809590915502892380935502F0
:10196000089510925502089590915402892B809306
:1019700054020895809590915402892380935402D3
:1019800008951092540208958091330208950895A5
:101990000C94C70C0C94C80C9091AD0292FD08C039
:1019A00090913302981721F0809333020C94CA0C63
:1019B000089580913302882329F01092330280E049
:1019C0000C94CA0C0895CF93DF93E0910201F0913B
:1019D0000301809155028083E0910201F09103019F
:1019E000908180915402892B8083809133028823D7
:1019F00081F0E0910201F09103019081892B8083B5
:101A000080910201909103010E94F41981110E94BA
:101A1000D90CC0910201D091030140E250E062E193
:101A200072E0CE010E941A23892B69F080E2FE0148
:101A3000A2E1B2E001900D928A95E1F7CE01DF912B
:101A4000CF910C94A019DF91CF9108950C94C70CFD
:101A50009091AD0292FD10C098E0899F90011124F1
:101A6000262B209332020E9406088091320285952F
:101A7000859585950C94260D0C94060810923202DB
:101A800080E00C94260D2091320280958223809371
:101A90003202982F977099F430E0482F082E000CEE
:101AA000550B2417350759F09091AD0292FD07C0F0
:101AB0008595859585950E9427080C943E0D08957F
:101AC0009091AD0292FB222720F9281769F080FB44
:101AD00092F99093AD028091AC029091AD020E9478
:101AE000AE0D82E00C94430D08958091AD0282FB0F
:101AF000882780F991E089270C94600D81E00C948F
:101B0000600D80E00C94600D6FEF7FEF80E090E05F
:101B10000C94532380E090E00E942F2321E0893E23
:101B20009E4F09F020E0822F089582E090E00C940F
:101B3000272383E090E00C942723CF9384E090E068
:101B40000E942723C82F82E290E00E9427232C2F97
:101B500030E0A901582BCA01CF910895CF93C92F26
:101B6000682F84E090E00E9435236C2F82E290E0A1
:101B7000CF910C943523AB01BC018FE090E00C9425
:101B80004723AB01BC0183E190E00C94472360E064
:101B900070E0CB010C94C10D60E070E0CB010E94BD
:101BA000BB0D0C94C70D69EE7EEF80E090E00E94C3
:101BB000532360E082E090E00E94352360E083E000
:101BC00090E00E9435231092D6011092D701109216
:101BD000D8011092D90160E084E090E00E943523A2
:101BE00060E082E290E00E94352360E085E090E0D2
:101BF0000E94352360E086E090E00E9435236FEF7D
:101C000087E090E00E94352340E050E0BA0188E090
:101C100090E00E94472360E08DE090E00E94352331
:101C200040E050E0BA0188E190E00E94472360E084
:101C300087E190E00E94352340E050E0BA018CE15A
:101C400090E00E94472360E070E080E290E00E9414
:101C5000532340E050E0BA0188E190E00E9447231E
:101C60000C94CC0D0C94D30D682F8EE090E00C9466
:101C700035230E945A1B609366027093670280931B
:101C8000680290936902609362027093630280938A
:101C9000640290936502089585B7806885BF85B713
:101CA000806885BF089581E008950C94530E0895CF
:101CB0000C94570E0C94570E0C945A0E0C94570E0D
:101CC0000C945E0E0C94570E0E944C0E88E291E12B
:101CD0000E948A190E94620E0C94600E0E94580E97
:101CE0000C94570E0E9442110E9407030C943C175B
:101CF0000E94451B0E9427120E94720E0E947515B9
:101D00000C945C0E5F926F927F928F929F92AF9233
:101D1000BF92CF92DF92EF92FF920F931F93CF93D8
:101D2000DF93CDB7DEB72A970FB6F894DEBF0FBEAC
:101D3000CDBF0E943C12C82E81110E94390E36E59B
:101D4000832E32E0932E00E010E0502E802F0E9470
:101D500066115C01F401619071904F01682679264B
:101D600061147104B1F40F5F1F4F0630110569F75C
:101D70008FEF89838A831B820E944E1B8160782F9C
:101D80009D838C8349815A816B818D810E942903B7
:101D90003AC080916A0281FD0E946F11D12CEE241D
:101DA000E394F12CC3018E219F21892B29F10E94FC
:101DB000550E8823A9F0DE825F82AE20BF2081E02D
:101DC000AB2809F480E088870E944E1B8160782F41
:101DD0009A8789874E815F8168858A850E94290359
:101DE000000F111FF801EA5AFD4F80819181E8260A
:101DF000F926F182E08207C0D394EE0CFF1CF0E1DB
:101E0000DF12D0CFB0CF81E0C11001C080E02A96B0
:101E10000FB6F894DEBF0FBECDBFDF91CF911F91FB
:101E20000F91FF90EF90DF90CF90BF90AF909F9079
:101E30008F907F906F905F9008950E94820E0E9415
:101E40003B170E9443140C941E03CF93DF930E9410
:101E50005110EC01811521E5920708F045C081156C
:101E600030E5930708F094C0883E910528F5803E40
:101E7000910508F0F8C0883A910570F4853A91050B
:101E800008F07CC08130910509F475C008F4E8C001
:101E9000049708F0E8C0E4C08F3B910508F0E0C06B
:101EA000C85AD0E0CC0FDD1FC65BDE4F0990D88149
:101EB000C02DCE019464D8C0811540E2940758F437
:101EC000811551E0950708F0CEC08D3E910508F4CC
:101ED000C7C09065C9C0C11580E4D80708F4C0C068
:101EE000DF70CE01906AC0C0811525E59207A8F485
:101EF000811534E5930708F095C0811543E59407F3
:101F000008F07BC0811552E5950708F061C0D82F15
:101F1000CC27CE01816F906AA7C0C11589E5D8078B
:101F2000A0F4C11528E5D20708F082C0C11536E536
:101F3000D30708F095C08C2F0E94E5108F7190E0B8
:101F4000D82FCC27CE0190628FC0C1154AE5D407A7
:101F500008F474C0CE0190568115904208F080C0FC
:101F60008D2F8F710E94E510DD27D0628F71AE0139
:101F7000582BCA0179C081E090E076C0C55AD0E004
:101F8000C858DE4F8881C82FD0E0CE0190646CC065
:101F900074E0969587957A95E1F7282F23703C2F6A
:101FA000337081E090E002C0880F991F3A95E2F704
:101FB0009C68AC01522B9A019C2F9F709695969528
:101FC00050E2959FE0011124C9018C2B9D2B4CC040
:101FD0008370992721E030E002C0220F331F8A95D9
:101FE000E2F79C2F9695969580E2989FE001112448
:101FF000C22BD32BCE019C6837C08370992721E078
:1020000030E002C0220F331F8A95E2F79C2F96958D
:10201000969540E2949FE0011124C22BD32BCE0170
:102020009A6822C0D82FCC27CE01846F906A1CC03A
:10203000DC2FCC27CE01806F906A16C08C2F8F705A
:102040000E94E51094E0D695C7959A95E1F7CF7078
:10205000D0E0DC2FCC27D0699E01282BC90104C019
:1020600080E090E001C0CE01DF91CF910895E72F8D
:10207000F0E096E0899FE00DF11D112484E0EE0F61
:10208000FF1F8A95E1F7E60FF11DEE0FFF1FE852E3
:10209000FF4F8591949108950E9437100E94250F5B
:1020A00008958238910569F1B0F48133910509F4FE
:1020B0006DC048F48932910509F463C08A329105F4
:1020C00009F469C008958533910509F455C0893331
:1020D0009105B9F00895833E910569F138F4803E89
:1020E0009105B1F0823E910509F10895863E910572
:1020F000A9F1873E9105B9F1843E910509F064C0CC
:1021000023C02091AC0220FD4FC021FD4DC0089599
:102110008091AC0280FD44C08091AD0280FF44C03C
:102120008091AC0284FD42C083EE4DC08091AC0230
:1021300082FF38C0F5CF8091AC0282FD33C0809120
:10214000AD0280FD31C0ECCF8091AD0281FF32C085
:102150008091AC0284FD2AC087EE35C08091AC022C
:1021600083FF26C0F5CF8091AC0283FD21C0809112
:10217000AD0281FD1FC0ECCF8091AC0285FD1CC07B
:102180001DC08091AC0285FD19C016C08091AC02C3
:1021900086FD16C017C08091AC0286FD13C010C02A
:1021A00089E311C082EE0FC080EE0DC080E00BC04D
:1021B00086EE09C084EE07C089E205C085E303C04E
:1021C0008AE201C081E390E008959091AC0292FF11
:1021D0000DC0282F2871283019F4877F846006C02D
:1021E000282F2471243011F48B7F886093FF0DC059
:1021F000282F2871283119F4877E846106C0282F82
:102200002471243111F48B7E88612091AD0220FF6E
:102210000DC0382F3871383019F4877F816006C0BF
:10222000382F3171313011F48E7F886021FF0DC05D
:10223000282F2871283119F4877E816106C0282F44
:102240002171213111F48E7E886194FD877E08957D
:1022500080E008950C94840D0E943C128FE39CE969
:102260000197F1F700C000000E943C1280E00E943C
:10227000661180FF04C00E942A110C949B1B0895D4
:102280000C942C110E948A0D811102C00E94320E02
:102290000E94950D80936A020E949D0D9093AD025D
:1022A0008093AC020E9440110E94990D682F70E04B
:1022B00080E090E00E94A6076091D2017091D30166
:1022C0008091D4019091D5010C94DE07E82FF0E0C5
:1022D000EE0FFF1FE654FD4F808191810895089510
:1022E00080EA8A95F1F7089500C008950C94701162
:1022F00008950C9478110C9479110C9478110C9425
:102300007D11F894E82FE295EF70F0E031A1282FCD
:102310002F7081E090E001C0880F2A95EAF7982F8E
:102320009095932391A392A1892B82A378940895E9
:102330000F931F93CF93DF93CBE8D1E089918F3F29
:1023400011F00E94811181E0C139D807B9F7CBE7BC
:10235000D1E00BE811E089918F3F11F00E948111CB
:102360000C171D07C1F7DF91CF911F910F910895B1
:10237000BF92CF92DF92EF92FF920F931F93CF9372
:10238000DF938C01C62FD0E0CE0185579E4F6C01A4
:10239000FC0190819F3F09F450C0B62EF894E92FBC
:1023A000E295EF70F0E081A19F7021E030E001C084
:1023B000220F9A95EAF7822B81A382A120952823E8
:1023C00022A378940E947411EBE7F1E04BE851E00E
:1023D00021E030E0E12CF12C61916F3F89F0A62FD4
:1023E000A295AF70B0E090968C9190E06F7002C0B3
:1023F000959587956A95E2F780FD02C0C90102C0F4
:1024000080E090E0E82AF92A220F331F4E175F0779
:1024100019F7F60180818F3F11F00E94811161E070
:10242000E114F10409F460E08B2D0E947611CC0FC9
:10243000DD1FC00FD11FF982E882DF91CF911F917C
:102440000F91FF90EF90DF90CF90BF9008950E9482
:1024500098118CE0EAEBF2E0DF01982F1D929A953B
:10246000E9F7EEEAF2E0DF011D928A95E9F786E0EE
:102470000E9487120C947002FF920F931F93CF93C8
:10248000DF93CDB7DEB72C970FB6F894DEBF0FBE43
:10249000CDBF8E010F5F1F4F8CE0F80111928A951E
:1024A000E9F7F12C6F2DC8010E94B811F394F6E002
:1024B000FF12F8CF4CE050E0B8018EEA92E00E94A3
:1024C0001A23FF24F394009709F4F12C892B41F08F
:1024D0008CE0F801AEEAB2E001900D928A95E1F746
:1024E0002F2D46E06AEB72E08EEA92E00E9488129D
:1024F0000E9472028F2D2C960FB6F894DEBF0FBE8D
:10250000CDBFDF91CF911F910F91FF900895089556
:10251000FF920F931F93CF93DF93F82E092F162F5F
:10252000D72FC42F222349F081E080936D020E94AF
:102530004E1B90936C0280936B0280916D028823F6
:10254000D9F080916B0290916C020E94661B0597F6
:1025500098F0EF2DF02FA12FBD2F80E090E04C2FB1
:1025600050E08417950734F4219131912D933D93D8
:102570000196F7CF10926D02DF91CF911F910F91CD
:10258000FF9008950E94661D0E94780E0C94721DA3
:102590000E94761D0E941D0F0C94901D0E94EC1A43
:1025A0000E944D1D0E94640E0E94C2120E94C81219
:1025B0000E946E0EFBCF8091740280FF06C0609176
:1025C000090170E0660F771F26C081FF04C060918B
:1025D000090184E005C082FF07C06091090188E01D
:1025E000689FB001112417C0909173029923D1F014
:1025F00060910801961788F72091090188E0289FCB
:1026000090011124929FA001939F500D112470E01E
:10261000CA010E94C4226038710540F46115710539
:1026200019F406C068E070E0862F08958FE70895DA
:1026300081E008958091740280FF08C060910501D7
:1026400070E0759567957595679521C081FF06C007
:102650006091050170E07595679519C082FF04C00F
:102660006091050170E010C090917202992399F079
:10267000609104019617A0F780910501899FC00120
:10268000112470E00E94C4226038710540F4611585
:10269000710519F406C061E070E0862F08958FE798
:1026A000089581E008958D3E21F40E94DB1281950A
:1026B00004C08E3E29F40E94DB12809378020895B4
:1026C0008F3E21F40E94DB12819504C0803F29F4E3
:1026D0000E94DB12809377020895893F19F40E94CB
:1026E0001A1305C08A3F31F40E941A138195809312
:1026F000790208958B3F21F40E941A13819504C03A
:102700008C3F29F40E941A1380937A0208959FE067
:10271000980F983078F421E030E0A90102C0440F0E
:10272000551F9A95E2F7CA0190917602892B809302
:10273000760208958D3F21F48091740281600BC070
:102740008E3F21F480917402826005C08F3F29F48E
:102750008091740284608093740208958D3E39F4F0
:102760009091780297FF35C01092780259C08E3E42
:1027700029F4909178021916BCF32BC0909177023E
:102780008F3E29F497FF25C01092770249C0803F01
:1027900019F41916CCF31DC090917902893F29F4E0
:1027A0001916BCF4109279023BC08A3F19F497FFC6
:1027B00010C0F8CF8B3F39F490917A0297FF09C08F
:1027C00010927A022DC08C3F21F490917A02191652
:1027D000BCF39FE0980F983080F421E030E0A9012D
:1027E00002C0440F551F9A95E2F7CA018095909157
:1027F000760289238093760213C08D3F21F4809165
:1028000074028E7F0BC08E3F21F4809174028D7F05
:1028100005C08F3F29F4809174028B7F80937402EE
:1028200080917702811106C080917802811102C0E7
:102830001092730280917902811106C080917A0210
:10284000811102C01092720208950E944E1B2091C5
:102850007702211104C020917802222321F0909365
:1028600071028093700220917902211104C020919D
:102870007A02222321F090936F0280936E0285E703
:1028800092E00C94BA19EF92FF920F931F93CF939B
:10289000DF9300D000D000D0CDB7DEB786E0E5E70B
:1028A000F2E0DE01119601900D928A95E1F7E09039
:1028B0007702F09078020091790210917A021092DA
:1028C0007702109278021092790210927A02E11047
:1028D00003C0FF2009F45DC08091700290917102E5
:1028E0000E94661BAC0190917302992339F02091EC
:1028F0000A0130E02417350758F04BC020910B0136
:102900008AE0289F900111242417350718F041C050
:102910009F3F19F09F5F90937302EE2061F00E9439
:10292000DB121E1414F09FEF01C091E0989F902DD0
:10293000112490937702FF2061F00E94DB121F1494
:1029400014F09FEF01C091E0989F902D1124909377
:102950007802309177023323E1F02091780222232C
:10296000C1F045EB3403C0011124992319F0909371
:10297000770203C081E08093770235EB2303C00127
:102980001124992319F09093780203C081E0809379
:102990007802011103C0112309F45DC080916E0219
:1029A00090916F020E94661BAC0190917202992374
:1029B00039F02091060130E02417350758F04BC05C
:1029C000209107018AE0289F9001112424173507E0
:1029D00018F041C09F3F19F09F5F9093720200234F
:1029E00061F00E941A13101614F09FEF01C091E0DD
:1029F000989F902D112490937902112361F00E94E9
:102A00001A13111614F09FEF01C091E0989F902DBA
:102A1000112490937A02309179023323E1F02091CE
:102A20007A022223C1F045EB3403C001112499231B
:102A300019F09093790203C081E08093790235EB1D
:102A40002303C0011124992319F090937A0203C043
:102A500081E080937A028091770281110BC080918E
:102A60007802811107C080917902811103C08091A1
:102A70007A0281110E942514EB82FC820D831E8351
:102A800086E0FE013196A5E7B2E001900D928A95AD
:102A9000E1F726960FB6F894DEBF0FBECDBFDF91EB
:102AA000CF911F910F91FF90EF900895E5E7F2E02D
:102AB00086E0DF011D928A95E9F710927302109269
:102AC000720210927402089586E090E00C9427231D
:102AD000682F86E090E00C9435238091C6028470C4
:102AE00089628093C6020C9468150E948A0D811138
:102AF00004C00E94320E0E946D150E9464158093DE
:102B0000C602282F26952695269530E026303105D9
:102B100024F0877088628093C6028091C60280FF8D
:102B200004C086958695869501C080E00C94861633
:102B30002091C602822F869586958695482F50E073
:102B40004530510554F48F5F982F990F990F990FC5
:102B5000822F8770892B8093C6028091C602816084
:102B60008093C6020E9468158091C602869586955C
:102B700086950C9486168091C602982F9695969508
:102B80009695A1F0915E990F990F990F8770892BF7
:102B90008093C602887F91E009F490E08091C6029C
:102BA00090FB80F98093C6020E9468158091C6024E
:102BB0008695869586950C9486168091C60280FD32
:102BC00013C081608093C602813019F489E080933C
:102BD000C6028091C6020E9468158091C602869541
:102BE000869586950C94861608958091C60280FF7E
:102BF00008C08E7F8093C6020E94681580E00C9406
:102C0000861608958091C60280FD0C94F5150C94EB
:102C1000DD159091C602892F8695869586958F5FE2
:102C20008F719770863038F4880F880F880F892B42
:102C30008093C60202C09093C6028091C602887F2C
:102C400091E009F490E08091C60290FB80F98093B6
:102C5000C6020E9468158091C60286958695869563
:102C60000C948616863008F085E09091C602977025
:102C7000282F220F220F220F922B9093C602987FAB
:102C800021E009F420E09091C60220FB90F9909396
:102C9000C6020C9486160E9432168091C6020C94CD
:102CA00068159C01FB018281882349F12E3BFCE5DC
:102CB0003F07C9F040F42C3BECE53E0769F02D3BA3
:102CC0003C4561F00895203C9CE5390791F070F097
:102CD000213C3C4589F0089585E001C080E00E94D8
:102CE0004B1680E008950E94BB15FBCF0E949815FB
:102CF000F8CF0E940216F5CF0E940916F2CF81E0AC
:102D00000895269A2E9808952E9808958F929F924E
:102D1000AF92BF92CF92DF92EF92FF920F931F93E9
:102D2000CF93DF93C82F863050F4811109C0809172
:102D300080008F7D809380000E94841606C0C5E0CD
:102D400080918000806280938000A0918600B09185
:102D500087002C2F30E00E94002325E030E040E087
:102D600050E00E94D8220027122F232F342F012F4A
:102D7000122F232F332780918600909187006CE0DB
:102D800070E00E94B0226017710730F0C80169E05E
:102D900070E00E94B0225EC0809186009091870012
:102DA000E0908600F0908700E0918600F091870027
:102DB000C6E0D0E0BE010E94B022060F171F211D01
:102DC000311D4801590185E0880C991CAA1CBB1CC7
:102DD0008A95D1F7C701BE010E94B0226F01E12C94
:102DE000F12CA7019601260F371F411D511DC5016A
:102DF000B4010E94D82269017A01E0918600F09125
:102E00008700CA01B9010E94A0229B01AC01DF0129
:102E10000E940F239B01AC01C701B6010E94A022B2
:102E2000DC01CB012FE0B695A795979587952A955C
:102E3000D1F7009186001091870020E030E008175C
:102E400019072A073B0728F46091860070918700D4
:102E5000CB01BC0170938B0060938A00DF91CF910E
:102E60001F910F91FF90EF90DF90CF90BF90AF90A8
:102E70009F908F90089508950E94811682E280931A
:102E8000800089E1809381008FEF9FEF909387000E
:102E9000809386000C947515CF93DF93EC01FB01B2
:102EA0008281882309F43CC1C430FDE5DF0760F46A
:102EB000CB3F9CE5D90788F49E0122503C45243144
:102EC000310508F02EC109C0C236EDE5DE0729F054
:102ED000C63AFDE5DF0709F024C10E949D0D9093DD
:102EE000AD028093AC02C1318CE5D80709F4C6C0AD
:102EF00008F042C0C930ECE5DE0709F49BC000F5DC
:102F0000C5308CE5D80709F485C078F4C330ECE50A
:102F1000DE0709F478C008F07AC0C230DC4509F059
:102F2000F5C08091AC028160EFC0C7309CE5D90745
:102F300009F478C008F07AC08091AC028061E4C0E6
:102F4000CD30FCE5DF0709F487C058F4CB309CE5B1
:102F5000D90709F479C008F07BC08091AC02886081
:102F60006FC0CF30FCE5DF0709F480C008F082C0F5
:102F70008091AC02877FC8C0CE3F9CE5D90709F499
:102F800071C000F5C531FCE5DF0709F485C068F4C0
:102F9000C3319CE5D90709F475C008F095C00E94BB
:102FA0004E078091AC028F77AFC0CC3FFCE5DF07C6
:102FB000A9F108F054C0CB3FDC4509F0A7C08091CF
:102FC000AD0240C0C230EDE5DE0709F489C058F417
:102FD000C1158DE5D80709F45AC008F069C0809181
:102FE000AD0282602FC0C236EDE5DE0709F47CC079
:102FF000C63AFDE5DF0709F481C0C330DD4509F0BD
:1030000085C080E06EC08091AC0282607DC08091FE
:10301000AC0216C08091AC02886076C08091AD028F
:1030200082604FC08091AC0280626EC08091AC0221
:1030300080646AC00E944E078091AC02806864C0C0
:10304000846062C081603DC08091AC028E7F5CC0B4
:103050008091AC028D7F58C08091AC0216C08091E7
:10306000AD0218C08091AD028D7F2BC08091AC0263
:103070008F7E4AC08091AC028F7D46C08091AC02A9
:103080008F7B42C08091AC02877F8B7F3DC0809157
:10309000AD028D7F8E7F15C08091AC0282FB22270E
:1030A00020F991E0922790FB82F990FB83F92CC0E4
:1030B0008091AD02982F909591708E7F892B90FB17
:1030C00081F98093AD0222C00E944E078091AC022C
:1030D00087FB222720F991E0922790FB87F914C003
:1030E00081E00E94340E12C08091AC0284FB222742
:1030F00020F991E0922790FB84F906C08091AC0200
:10310000982F909590FB80F98093AC028091AC024F
:103110009091AD020E94AE0D0E944E0780E001C06A
:1031200081E0DF91CF910895CF93DF9386319C4565
:1031300041F5EB010E94A10C982F8A812091020198
:1031400030910301882379F09A7A81E009F480E0D4
:1031500080937B02911102C069E201C065E3C9015D
:103160000E948A1A0AC080917B02811102C069E222
:1031700001C065E3C9010E94951A0E94E30C80E03A
:1031800001C081E0DF91CF9108950F931F93CF93FA
:10319000DF93C42FD22FFC0182818823C9F0409392
:1031A0007E020E944E1B90937D0280937C0280E2FF
:1031B0008C0F883008F057C0C77081E001C0880FBD
:1031C000CA95EAF7DF91CF911F910F910C94AB0450
:1031D00080917E02481330C080917C0290917D02E4
:1031E0000E94661B883C910538F510E21D0FCD1733
:1031F000B9F080E28C0F883040F4C77081E001C0E4
:10320000880FCA95EAF70E94B204183028F581E0C9
:103210009D2F977001C0880F9A95EAF70E94AB0422
:10322000802F0E94A2041830F0F4D77081E001C012
:10323000880FDA95EAF70AC080E28C0F883098F49C
:10324000C77081E001C0880FCA95EAF7DF91CF917E
:103250001F910F910C94B204802FDF91CF911F9199
:103260000F910C94A204DF91CF911F910F910895BB
:103270000F939C01CB01243F4CE5340731F188F4D6
:10328000293DFCE53F07D9F02A3D4CE5340779F1AB
:10329000283D3C45A9F506E221EE41EE68ED7CE5CE
:1032A0002BC0263FFCE53F07E1F0A8F0273F3C4557
:1032B00039F507E225EE46EE67EF7CE51DC007E233
:1032C00025EE45EE69ED7CE517C006E221EE40EE05
:1032D00064EF7CE511C007E225EE44EE65EF7CE586
:1032E0000BC006E221EE42EE66EF7CE505C008E287
:1032F00021E045EE6AED7CE50E94C51880E008C03B
:10330000FC018281882319F010927E0201C081E0C5
:103310000F91089590939301809392010895909353
:103320008402809383020895E0918302F0918402E5
:10333000309721F00190F081E02D099480E008950C
:10334000E0918302F0918402309799F02091180166
:10335000222359F02091AC0227FF07C0DC012C91F9
:1033600011962C93119726E02C930280F381E02D87
:1033700009940895E0918302F0918402309739F026
:1033800022E0DC012C930480F581E02D099408955E
:1033900020918102309182022817390771F09093B1
:1033A000820280938102E0918302F091840230973F
:1033B00021F00680F781E02D0994089520917F0285
:1033C000309180022817390771F090938002809322
:1033D0007F02E0918302F0918402309721F0008413
:1033E000F185E02D09940895FC0132968091180131
:1033F000882331F08091AC0287FF02C09EE101C0BA
:1034000096E080E0915028F021912223D9F38F5F3C
:10341000F9CF0895662351F1209118012223E9F094
:103420002091AC0227FF19C0462F46954695469538
:103430004E31E0F4677021E030E002C0220F331F0C
:103440006A95E2F7FC01E40FF11D828190E02823E8
:10345000392381E0232B69F409C0FC0132960896D8
:103460002191621729F0E817F907D1F780E0089554
:1034700081E008959C01FC0132969FEF80E041912C
:10348000461789F09F3F19F4411101C0982F8F5FB3
:103490008630A9F79F3F39F0F901E90FF11D97FD3B
:1034A000FA956283089508959C012A5F3F4FFC01BD
:1034B0004281461301C01282019682179307B9F721
:1034C0000895262F2695269526952E3168F4FC0121
:1034D000E20FF11D677021E030E001C0220F6A9514
:1034E000EAF78281282B22830895262F2695269598
:1034F00026952E3170F4FC01E20FF11D677021E07A
:1035000030E001C0220F6A95EAF7209582812823D6
:103510002283089520911801222329F02091AC02E2
:1035200027FD0C94611A0C943A1A20911801222359
:1035300029F02091AC0227FD0C94751A0C94541AB2
:1035400020911801FC013296222331F08091AC02C7
:1035500087FF02C08EE101C086E0DF011D928A95DF
:10356000E9F7089508950C94B21A83E080938502D8
:103570000C94B31A811102C081E001C082E08093F3
:1035800085020C94B31A0C94BA1A81E080938502D8
:103590000C94B31A0C94C51A08950C94CC1A0C947C
:1035A000CD1A0C94CC1A0C94CC1A0C94CC1ACF9340
:1035B0000E94D31A0E943C120E94D11AC0E08C2FA4
:1035C0000E946611892B29F4CF5FC630C1F780E0D5
:1035D00001C081E0CF91089508951F920F920FB618
:1035E0000F9211248F939F93AF93BF938091860284
:1035F000811113C08091C7029091C802A091C902A5
:10360000B091CA024196A11DB11D8093C70290934B
:10361000C802A093C902B093CA02BF91AF919F9113
:103620008F910F900FBE0F901F9018958091CF0231
:10363000843031F10E94DD021092860220E488E19C
:1036400090E00FB6F894A895809360000FBE209389
:10365000600083B7817F846083BF83B7816083BF4D
:103660007894889583B78E7F83BF0FB6F894A8951A
:1036700080916000886180936000109260000FBEAE
:1036800008950E944E070C94E40282E084BD93E00A
:1036900095BD9AEF97BD80936E0008952FB7F8946B
:1036A0008091C7029091C802A091C902B091CA024C
:1036B0002FBF08952FB7F8946091C7027091C80288
:1036C0008091C9029091CA022FBF08959C014FB703
:1036D000F8948091C7029091C802A091C902B0915C
:1036E000CA024FBF821B930B089578941F920F92CA
:1036F0000FB60F9211248F939F93AF93BF93809136
:10370000C7029091C802A091C902B091CA02019665
:10371000A11DB11D8093C7029093C802A093C90256
:10372000B093CA02BF91AF919F918F910F900FBE3E
:103730000F901F90189581E08093E00080E28093C5
:10374000D8001092C9008FE19EE40197F1F700C004
:10375000000087E090EBDC018093D8029093D902BF
:10376000A093DA02B093DB029CE088E10FB6F894F4
:10377000A895809360000FBE90936000FFCF80916A
:10378000AA020895089522E02093E9002FEF3091D6
:10379000E800215035FD06C035ED3A95F1F70000FF
:1037A0002111F5CF2091E80025FF0BC040E050E04B
:1037B00066E070E00E94021E8091E8008E778093A0
:1037C000E8000895CF93DF9320911801222339F068
:1037D0002091AC0227FF03C060E222E002C068E053
:1037E00021E02093E9002FEF3091E800215035FDD2
:1037F00006C035ED3A95F1F700002111F5CF209183
:10380000E80025FF1DC0EC0180911801811105C061
:1038100040E050E068E070E003C070E040E050E05D
:10382000CE010E94021E8091E8008E778093E8000E
:1038300080E2FE01AAE8B2E001900D928A95E1F7DC
:10384000DF91CF91089580938702709389026093EE
:1038500088028091CF02843001F582E08093E900F4
:103860008FEF9091E800815095FD06C095ED9A95F7
:10387000F1F700008111F5CF8091E80085FF0DC0C0
:1038800040E050E063E070E087E892E00E94021EB2
:103890008091E8008E778093E8000895BC0184E071
:1038A0000C94231CBC0183E00C94231C8091CE0259
:1038B000811109C00E94931F0E94F01F8091E200B5
:1038C00084608093E20008951092CE0208950C94D3
:1038D000CA1A6091CB0281E0611101C080E00C94B2
:1038E000B51A9091CF0281E0943009F080E06091A8
:1038F000CB020C94BA1A42E061EC81E00E940C1FEA
:1039000042E261EC82E00E940C1F9091CF0281E0C4
:10391000943009F080E06091CB020C94C31A80913E
:10392000D102833009F461C030F4813071F082300B
:1039300009F49AC008958A3009F486C08B3009F4DE
:103940006CC0893009F0A8C020C08091D002813AB3
:1039500009F0A2C08091E800877F8093E800809101
:10396000D4029091D502892B21F460E28AE892E09A
:1039700003C060E080E090E070E00E944D1E809106
:10398000E8008B778093E80008958091D00281321F
:1039900009F082C08091D4029091D502029708F07C
:1039A0007BC08091E800877F8093E8008091E800E9
:1039B00082FD05C08091CF028111F8CF6DC02091AA
:1039C000F3008091F20090E0922B029731F4809105
:1039D000F100813011F0863021F48091F100809364
:1039E000AA028091E8008B7753C08091D002813A7F
:1039F00009F052C08091D4029091D502892B09F030
:103A00004BC08091E800877F8093E8008091E800B8
:103A100080FFFCCF8091180136C08091D0028132A6
:103A2000D9F58091D4029091D502892BA9F5809186
:103A3000E800877F8093E8000E94411F8091D202B6
:103A4000809318010C944E078091D002813221F5A9
:103A50008091E800877F8093E8000E94411F809159
:103A6000D3028093AB0208958091D002813AA1F4F1
:103A70008091E800877F8093E8008091E80080FFD4
:103A8000FCCF8091AB028093F1008091E8008E77AB
:103A90008093E8000C94411F089584B7877F84BF0A
:103AA0000FB6F894A89580916000886180936000BB
:103AB000109260000FBE90E080E80FB6F8948093FB
:103AC0006100909361000FBE0C94C51A0E94931F71
:103AD0000E94F01FE2EEF0E08081846080837894A1
:103AE0000C9485228CE091E00C948F198091CF0288
:103AF0008530A9F48091CF02853079F40E94161B9D
:103B00008091CD028823B1F30E94D71A882391F3C4
:103B10000E94EC1D0E944E07EDCF0C94411B0895AE
:103B200008950C94931D292F332723303105C9F0B4
:103B300060F42130310581F02230310509F044C0B4
:103B40008BE390E024E832E043C021323105E1F01C
:103B50002232310549F138C082E190E02FEB32E0AA
:103B600037C099278130910549F028F0029761F517
:103B7000E8E5F2E005C0E0E8F2E002C0ECE6F2E0E1
:103B8000849190E09F0124C06115710541F061307E
:103B90007105D1F489E090E02FEA32E019C089E0A4
:103BA00090E026E932E014C06115710541F0613002
:103BB000710551F486EB90E021ED32E009C080E41C
:103BC00090E027E833E004C080E090E020E030E0BF
:103BD000FA0131832083089580E189BD82E189BDA6
:103BE00009B400FEFDCF8091D8008F7D8093D8006E
:103BF0008091E00082608093E0008091E00081FD90
:103C0000FCCF0895CF92DF92EF92FF920F931F9314
:103C1000CF93DF93EC018B017A010E94601F811129
:103C200033C0E114F10439F0F70180819181081B60
:103C3000190BC80FD91FC12CD12C0115110519F171
:103C40008091E80085FD16C08091E8008E77809312
:103C5000E800E114F10449F0F70180819181C80E78
:103C6000D91ED182C08285E00FC00E94601F8823C8
:103C700021F30AC089918093F10001501109FFEFEF
:103C8000CF1ADF0ADACF80E0DF91CF911F910F9139
:103C9000FF90EF90DF90CF9008952091D602309161
:103CA000D7022617370748F06115710539F42091BE
:103CB000E8002E772093E80001C0B901FC0120E064
:103CC0006115710579F18091CF028823F1F185307A
:103CD000F1F18091E80083FD3CC08091E80082FD15
:103CE0002EC08091E80080FFEBCF2091F3008091FF
:103CF000F20090E0922B6115710551F0883091052A
:103D000038F421912093F100615071090196F3CFAD
:103D100021E0089709F020E08091E8008E778093F9
:103D2000E800CECF2111CFCF0AC08091CF028823E7
:103D300061F0853061F08091E80083FD0AC08091D8
:103D4000E80082FFF2CF80E0089582E0089583E0EA
:103D5000089581E008952091D6023091D702261768
:103D6000370748F06115710539F42091E8002E7786
:103D70002093E80001C0B901FC0120E06115710544
:103D800091F18091CF02882309F440C0853009F475
:103D90003FC08091E80083FD3DC08091E80082FD36
:103DA0002FC08091E80080FFE9CF2091F30080913F
:103DB000F20090E0922B6115710559F08830910561
:103DC00040F424912093F1003196615071090196DD
:103DD000F2CF21E0089709F020E08091E8008E778B
:103DE0008093E800CBCF2111CCCF0AC08091CF02C5
:103DF000882361F0853061F08091E80083FD0AC07E
:103E00008091E80082FFF2CF80E0089582E008957B
:103E100083E0089581E00895982F973068F5909396
:103E2000E900981739F07091EC002091ED00509165
:103E3000F00003C0242F762F50E021FD02C09F5FC9
:103E4000ECCF3091EB003E7F3093EB003091ED00F2
:103E50003D7F3093ED003091EB0031603093EB000B
:103E60007093EC002093ED005093F0002091EE0051
:103E700027FDE5CF80E008958F708093E90081E011
:103E800008958091D00287FF11C08091E80082FDE3
:103E900005C08091CF028111F8CF11C08091E80058
:103EA0008B770BC08091CF02882349F08091E80086
:103EB00080FFF8CF8091E8008E778093E800089526
:103EC0002091E4003091E50095E64091EC00842FCC
:103ED000817040FF23C08091E80080FD1DC080916B
:103EE000CF02882399F0853099F08091EB0085FD11
:103EF00011C04091E4005091E5002417350729F3E3
:103F0000915011F09A01E1CF84E0089582E0089584
:103F100083E0089581E0089580E008954091E800ED
:103F200042FFDDCF08950E9401200E940920E0EEAB
:103F3000F0E0808181608083E8EDF0E080818F7720
:103F4000808319BCA7EDB0E08C918E7F8C9380812B
:103F50008F7E80831092CE0208950F931F93CF938C
:103F6000DF930E9401200E940920C8EDD0E08881E3
:103F70008F77888388818068888388818F7D888314
:103F800019BC1092CF021092CB021092CD02109267
:103F9000CC0200EE10E0F80180818B7F8083888165
:103FA0008160888342E060E080E00E940C1FE1EEC7
:103FB000F0E080818E7F8083E2EEF0E0808181609E
:103FC0008083808188608083F80180818E7F8083F8
:103FD000888180618883DF91CF911F910F9108952F
:103FE000E8EDF0E080818F7E8083E7EDF0E0808176
:103FF0008160808384E082BF81E08093CE020C9454
:10400000AD1FE8EDF0E080818E7F80831092E200AA
:1040100008951092DA001092E10008951F920F9215
:104020000FB60F9211242F933F934F935F936F938B
:104030007F938F939F93AF93BF93EF93FF93809161
:10404000E10082FF0BC08091E20082FF07C08091F7
:10405000E1008B7F8093E1000E9484228091DA004E
:1040600080FF1FC08091D80080FF1BC08091DA00C4
:104070008E7F8093DA008091D90080FF0DC080E1AF
:1040800089BD82E189BD09B400FEFDCF81E0809346
:10409000CF020E94561C05C019BC1092CF020E948C
:1040A000641C8091E10080FF19C08091E20080FFD4
:1040B00015C08091E2008E7F8093E2008091E20043
:1040C00080618093E2008091D80080628093D80064
:1040D00019BC85E08093CF020E94691C8091E100A9
:1040E00084FF30C08091E20084FF2CC080E189BD54
:1040F00082E189BD09B400FEFDCF8091D8008F7D9B
:104100008093D8008091E1008F7E8093E1008091C0
:10411000E2008F7E8093E2008091E20081608093D4
:10412000E2008091CB02882311F084E007C08091E7
:10413000E30087FD02C081E001C083E08093CF02ED
:104140000E94711C8091E10083FF29C08091E200F0
:1041500083FF25C08091E100877F8093E10082E0AA
:104160008093CF021092CB028091E1008E7F8093EA
:10417000E1008091E2008E7F8093E2008091E20076
:1041800080618093E20042E060E080E00E940C1FCA
:104190008091F00088608093F0000E94671CFF917E
:1041A000EF91BF91AF919F918F917F916F915F91AF
:1041B0004F913F912F910F900FBE0F901F90189528
:1041C0001F920F920FB60F9211242F933F934F938C
:1041D0005F936F937F938F939F93AF93BF93CF938F
:1041E000DF93EF93FF93C091E900CF708091EC00D3
:1041F000D82FD17080FDD0E81092E9008091F000B6
:10420000877F8093F00078940E9424211092E90027
:104210008091F00088608093F000CD2BCF70C09328
:10422000E900FF91EF91DF91CF91BF91AF919F9105
:104230008F917F916F915F914F913F912F910F904F
:104240000FBE0F901F9018951F93CF93DF93CDB79C
:10425000DEB7AA970FB6F894DEBF0FBECDBFE0ED74
:10426000F2E08091F100819322E0E83DF207C9F786
:104270000E948F1C8091E80083FF2EC18091D002A4
:104280009091D102492F50E04A30510508F024C1E5
:10429000FA01EE59FF4F0C94FA22803821F082384F
:1042A00009F01AC108C08091CC029091CD029923E7
:1042B00089F082600FC08091D4028F70873008F03F
:1042C0000BC18093E9008091EB0085FB882780F982
:1042D0001092E9009091E800977F9093E800809316
:1042E000F1001092F100D1C0282F2D7F09F0F4C009
:1042F000882319F0823061F0EFC08091D2028130C2
:1043000009F0EAC0933009F080E08093CD022EC01E
:104310008091D20281112AC08091D4028F702FEF38
:10432000280F263008F0D8C08093E9002091EB00D8
:1043300020FF1CC0933021F48091EB00806214C0F8
:104340009091EB0090619093EB0021E030E0A901A7
:1043500002C0440F551F8A95E2F74093EA0010927D
:10436000EA008091EB0088608093EB001092E900F6
:104370008091E800877F8093E8000E94411FACC0D5
:104380008111AAC01091D2021F778091E30080783A
:10439000812B8093E3008091E800877F8093E80081
:1043A0000E94411F8091E80080FFFCCF8091E300D4
:1043B00080688093E300111102C082E001C083E0B5
:1043C0008093CF0289C08058823008F085C08091E8
:1043D000D2029091D3028C3D53E0950779F583E0AA
:1043E0008A838AE289834FB7F894DE01139620E02E
:1043F0003EE051E2E32FF0E050935700E49120FFBC
:1044000003C0E295EF703F5FEF708E2F90E0EA30CF
:1044100010F0C79601C0C0968D939D932F5F2431F5
:1044200049F74FBF8091E800877F8093E8006AE2F8
:1044300070E0CE0101960E944D1E16C06091D4021C
:104440007091D502AE014F5F5F4F0E94911DBC017C
:10445000892B09F441C09091E800977F9093E80080
:1044600089819A810E94AB1E8091E8008B778093AE
:10447000E80032C0803881F58091E800877F809322
:10448000E8008091CB028093F1008091E8008E7764
:1044900072CF811121C08091D2029091D3029927CD
:1044A0000297D4F48091E800877F8093E8008091A0
:1044B000D2028093CB020E94411F8091CB028111D6
:1044C00006C08091E30087FD02C081E001C084E066
:1044D0008093CF020E947B1C8091E80083FF0AC07A
:1044E0008091E800877F8093E8008091EB008062F4
:1044F0008093EB00AA960FB6F894DEBF0FBECDBF37
:10450000DF91CF911F9108950895CF938091CF02AD
:104510008823A1F0C091E900CF709091EC00892F21
:10452000817090FD80E8C82B1092E9008091E8002E
:1045300083FD0E942421CF70C093E900CF9108959C
:10454000DB018F939F930E940F23BF91AF91A29F96
:10455000800D911DA39F900DB29F900D1124089581
:10456000AA1BBB1B51E107C0AA1FBB1FA617B70799
:1045700010F0A61BB70B881F991F5A95A9F78095B5
:104580009095BC01CD01089597FB072E16F4009479
:1045900007D077FD09D00E94B02207FC05D03EF479
:1045A000909581959F4F0895709561957F4F0895DF
:1045B000A1E21A2EAA1BBB1BFD010DC0AA1FBB1F27
:1045C000EE1FFF1FA217B307E407F50720F0A21B99
:1045D000B30BE40BF50B661F771F881F991F1A9406
:1045E00069F760957095809590959B01AC01BD0130
:1045F000CF010895EE0FFF1F0590F491E02D09946F
:10460000A29FB001B39FC001A39F700D811D112413
:10461000911DB29F700D811D1124911D08950E945E
:104620000023A59F900DB49F900DA49F800D911D18
:1046300011240895FB01DC0104C08D9101908019C3
:1046400021F441505040C8F7881B990B0895F999FF
:10465000FECF92BD81BDF89A992780B50895A8E153
:10466000B0E042E050E00C945B23262FF999FECF96
:1046700092BD81BDF89A019700B4021639F01FBAB5
:1046800020BD0FB6F894FA9AF99A0FBE08950396D2
:10469000272F0E9436230E943523252F0E94362380
:1046A000242F0C9436230196272F0E9436230C9436
:1046B0003523DC01CB01FC01F999FECF06C0F2BD28
:1046C000E1BDF89A319600B40D9241505040B8F7D0
:0646D0000895F894FFCFED
:1046D600C8003402280850011E0A1401BF1BE21B41
:1046E600C31B521C4E1CC21B01E200E900EA00B5C6
:1046F60000B600B700CD008301CC008A0192019478
:10470600012102230224022502260227022A02B3DD
:1047160000B4006F007000818283E200E900EA00C5
:10472600B500B600B700CD008301CC008A01920126
:1047360094012102230224022502260227022A02CC
:10474600B300B4006F007000818283F0F1C6676623
:10475600F59431303534979633F4F69091929395DB
:0247660037001A
:00000001FF
